:100000000C945D000C9485000C9485000C94850084
:100010000C9485000C9485000C9485000C9485004C
:100020000C9485000C9485000C9485000C9485003C
:100030000C9485000C9485000C9485000C9485002C
:100040000C9433010C9485000C94A3010C947D0155
:100050000C9485000C9485000C9485000C9485000C
:100060000C9485000C94850000000008000201003B
:100070000003040700000000000000000000000072
:10008000250028002B0000000000240027002A0083
:10009000040404040404040402020202020203032E
:1000A0000303030301020408102040800102040836
:1000B0001020010204081020322211241FBECFEFAD
:1000C000D8E0DEBFCDBF12E0A0E0B1E0EAE2FDE49F
:1000D00002C005900D92AA37B107D9F723E0AAE72D
:1000E000B2E001C01D92A533B207E1F710E0CDE503
:1000F000D0E004C02197FE010E946025CC35D107D5
:10010000C9F70E940D1E0C9493260C940000CF9208
:10011000DF92EF92FF920F931F93CF93DF936C01C7
:100120007A018B01C0E0D0E0CE15DF0581F0D80167
:100130006D918D01D601ED91FC910190F081E02D42
:10014000C6010995892B11F02196EECF7E01C701DA
:10015000DF91CF911F910F91FF90EF90DF90CF90A3
:100160000895089580E090E008950E9487268EE823
:1001700092E00E94060221E0892B09F420E0822F00
:100180000895EF92FF920F931F93CF93DF93EC01AB
:1001900081E0888F9B8D8C8D981305C0E889F98943
:1001A000808185FD26C0F62E0B8D10E00F5F1F4F5E
:1001B0000F731127E02E8C8DE8120CC00FB607FCD0
:1001C000FACFE889F989808185FFF5CFCE010E94B9
:1001D000B807F1CF8B8DFE01E80FF11DE35AFF4FF9
:1001E000F0829FB7F8940B8FEA89FB898081806247
:1001F0000AC09FB7F894EE89FF896083E889F9897E
:1002000080818370806480839FBF81E090E0DF9174
:10021000CF911F910F91FF90EF9008953FB7F89401
:100220008091840290918502A0918602B09187020C
:1002300026B5A89B05C02F3F19F00196A11DB11D41
:100240003FBFBA2FA92F982F8827820F911DA11D7C
:10025000B11DBC01CD0142E0660F771F881F991FB9
:100260004A95D1F708951F920F920FB60F9211245D
:100270002F933F938F939F93AF93BF93809180026F
:1002800090918102A0918202B091830230917F020D
:1002900023E0230F2D3720F40196A11DB11D05C0C9
:1002A00026E8230F0296A11DB11D20937F028093A3
:1002B000800290938102A0938202B0938302809186
:1002C000840290918502A0918602B09187020196E6
:1002D000A11DB11D8093840290938502A093860294
:1002E000B0938702BF91AF919F918F913F912F91D2
:1002F0000F900FBE0F901F9018951F920F920FB680
:100300000F9211242F933F934F935F936F937F939B
:100310008F939F93AF93BF93EF93FF938EE892E0F9
:100320000E94B807FF91EF91BF91AF919F918F917C
:100330007F916F915F914F913F912F910F900FBEE1
:100340000F901F9018951F920F920FB60F921124C5
:100350002F938F939F93EF93FF93E0919E02F091E1
:100360009F028081E091A402F091A50282FD12C05B
:1003700090818091A7028F5F8F732091A8028217CE
:1003800051F0E091A702F0E0E257FD4F958F809386
:10039000A70201C08081FF91EF919F918F912F91D2
:1003A0000F900FBE0F901F901895FC01538D448D38
:1003B000252F30E0842F90E0821B930B541710F010
:1003C000CF96089501970895FC01918D828D98171D
:1003D00061F0828DDF01A80FB11D5D968C91928D29
:1003E0009F5F9F73928F90E008958FEF9FEF089526
:1003F000FC01918D828D981731F0828DE80FF11DEF
:10040000858D90E008958FEF9FEF0895FC01918D09
:10041000228D892F90E0805C9F4F821B91098F7302
:100420009927089580E090E0892B29F00E94B70079
:1004300081110C9400000895DC01ED91FC9104847D
:10044000F585E02D6DE070E00994FC0197859F71C2
:1004500021F490899F7781E009F080E00895FC0104
:1004600097859F719D3029F490899F7781E0903521
:1004700009F080E008959B0177FF02C0295F3F4F9C
:1004800043E0359527954A95E1F7FC01E20FF31F0C
:10049000278530E0CB0168E070E00E943825A90193
:1004A00002C0559547958A95E2F7CA018170089573
:1004B000660F771F860F971FFC0182898058089569
:1004C000660F771F860F971FFC018189805808955A
:1004D000860F971FFC0181890895FC0114A60895D9
:1004E000FC0184A50895860F971F4195FC01418763
:1004F0000895860F971FFC01418708959B014423AF
:10050000E9F077FF02C0295F3F4F53E0359527950B
:100510005A95E1F7FC01E20FF31FCB0168E070E0B0
:100520000E94382521E030E0A90102C0440F551F88
:100530008A95E2F7CA019381892B1DC077FF02C01B
:10054000295F3F4F43E0359527954A95E1F7FC0138
:10055000E20FF31FCB0168E070E00E94382521E034
:1005600030E0A90102C0440F551F8A95E2F7CA0185
:1005700080959381892383830895660F771FFC01FB
:10058000E60FF71F8FE7489F402D11244058468300
:1005900008956F5F7F4F660F771FFC01E60FF71F0F
:1005A0008FE7489F402D1124405843830895660FDC
:1005B000771F860F971F4058FC01468308956F5F91
:1005C0007F4F660F771F860F971F4058FC014383AC
:1005D0000895FC01138280E8848385838683878362
:1005E0008087118612860895CF92DF92EF92FF9254
:1005F0000F931F93CF93DF938C01EB017A01DC0102
:1006000015968D919C9116978130910521F0029756
:1006100009F45DC014C0E881F9810288F389E02DF6
:10062000CB010995882331F082E090E0F8019683B0
:100630008583C3C1D80116961C921E921597D701C7
:10064000ED91FC91C284D384E881F9810084F18525
:10065000E02D60E070E0CE010995682F880F770BE0
:10066000880B990B0E941624AB01BC01C8010E94A3
:100670008F0D482F60E070E0C701F6010995D701A2
:10068000ED91FC91C484D584E881F9810284F385DD
:10069000E02D60E070E0CE010995682F880F770BA0
:1006A000880B990B0E941624AB01BC01C8010E9463
:1006B0008F0D482F60E070E0C701F601DF91CF9108
:1006C0001F910F91FF90EF90DF90CF900994D80188
:1006D0001396ED91FC9114973496EE0FFF1FE00FE7
:1006E000F11F4081518157FF02C04F5F5F4F559509
:1006F0004795D701ED91FC910284F385E02D60E0F0
:1007000070E0C7010995D8011396ED91FC911497FB
:100710003896EE0FFF1FE00FF11F4081518157FF08
:1007200002C04F5F5F4F55954795D701ED91FC9102
:100730000484F585E02D60E070E0C7010995E8814B
:10074000F9810288F389E02DCE010995882309F407
:100750004DC1F8018781E881F9810484F585E02D98
:10076000882309F461C062E070E0CE01099581112F
:1007700074C1E881F9810484F585E02D63E070E0BF
:10078000CE010995811169C1E881F9810484F5855B
:10079000E02D61E070E0CE01099581115EC1E88134
:1007A000F9810484F585E02D60E070E0CE010995C3
:1007B000811153C1E881F9810484F585E02D68E059
:1007C00070E0CE010995811148C1E881F981048466
:1007D000F585E02D69E070E0CE01099581113DC1FC
:1007E000E881F9810484F585E02D6AE070E0CE01AE
:1007F0000995811132C1E881F9810484F585E02DE4
:100800006BE070E0CE010995811127C1E881F98183
:100810000484F585E02D64E070E0CE010995811136
:100820001CC1F801178219C163E070E0CE0109957F
:100830008823C1F0D8011396ED91FC911497EE0F27
:10084000FF1FE00FF11F808591858230910514F024
:10085000019702C081E090E09187808781E0F801F4
:100860008783FBC0E881F9810484F585E02D62E08F
:1008700070E0CE0109958823A1F0D8011396ED917F
:10088000FC911497EE0FFF1FE00FF11F20853185BB
:1008900080899189019728173907F4F6C9010196D3
:1008A000DBCFE881F9810484F585E02D61E070E01B
:1008B000CE0109958823A1F0D8011396ED91FC9102
:1008C0001497EE0FFF1FE00FF11F208931898085FB
:1008D000918501968217930704F5C90101971DC000
:1008E000E881F9810484F585E02D60E070E0CE01B7
:1008F00009958823A9F0D8011396ED91FC911497DE
:10090000EE0FFF1FE00FF11F808991898F3F910546
:1009100014F4019602C08FEF90E0918B808B9ECFF4
:10092000E881F9810484F585E02D64E070E0CE0172
:100930000995882381F0D8011396ED91FC911497C5
:10094000EE0FFF1FE00FF11F118610868FE790E07A
:10095000918B808B47C0E881F9810484F585E02D77
:100960006BE070E0CE010995882321F0F801148234
:10097000138223C0E881F9810484F585E02D68E0C5
:1009800070E0CE010995882341F081E090E0D80124
:1009900014969C938E93139726C0E881F981048462
:1009A000F585E02D6AE070E0CE010995882339F0E5
:1009B00082E090E0F8019483838381E051CFE88165
:1009C000F9810484F585E02D69E070E0CE01099598
:1009D000882309F442C083E090E0D80114969C93E8
:1009E0008E93139781E017968C9337C080912B03D9
:1009F00090912C03892B61F17801B8E0EB0EF11C8A
:100A0000C0E0D0E0F7016081F2E0EF0EF11C8091D0
:100A10002B0390912C038C0F9D1F0E94F414809146
:100A20002B0390912C038C0F9D1FD70116966C9170
:100A300001960E94F4142296C830D10519F78091CE
:100A40002B0390912C03F801638108960E94F41403
:100A5000D80116961C921E921597DF91CF911F9187
:100A60000F91FF90EF90DF90CF9008956F927F925B
:100A70008F929F92AF92BF92CF92DF92EF92FF92AE
:100A80000F931F93CF93DF9300D000D0CDB7DEB785
:100A90008C01DC0191968C9191978111E1C088E0E5
:100AA000E4EBF1E01F9601900D928A95E1F7D801F1
:100AB000AE58BF4F80E090E067E070E041E050E06A
:100AC0009C0127703327FB01E21BF30B3A0102C0A4
:100AD000660C771CEA95E2F79301FC0133E0F5958B
:100AE000E7953A95E1F7E00FF11F378523232D9322
:100AF00001968034910521F7780162E2E60EF11C3F
:100B000080E4D7011D928A95E9F71C8261E0CE014D
:100B100004960E949F0C6AE070E0C7010E944A0D93
:100B2000C8018E549F4F2AE0FC0111922A95E9F7E3
:100B30004701F70140E050E077E0C72ED12CA191AA
:100B40009A0163E0359527956A95E1F7200F311FEB
:100B5000590162EBA60EB11C61E070E0A11102C068
:100B600060E070E0DA01A770BB2736016A1A7B0AE1
:100B700001C0660F6A94EAF7D901AE54BF4F2C91B9
:100B8000622BD5016C934F5F5F4F40355105B9F62D
:100B9000FC01208121110AC0F801ED54FF4F208192
:100BA000211104C031962081222329F081E0D8014F
:100BB00091968C9306C04AE050E063E071E00E9499
:100BC0008C268AE0E0E5F1E0D801579601900D927D
:100BD0008A95E1F780E5F70111928A95E9F781E4BA
:100BE000898361E0CE0101960E949F0C6AE070E06B
:100BF000C7010E944A0D019779F58AE0F8017796BE
:100C0000DF011D928A95E9F720E030E047E050E0EF
:100C1000F40161914F01F90193E0F595E7959A95FB
:100C2000E1F7E00FF11F81E090E0611102C080E088
:100C300090E0B901677077273A01661A770A01C018
:100C4000880F6A94EAF79789892B878B2F5F3F4F2C
:100C500020353105E9F6BDC0D80191961C92B9C086
:100C60007801B2E2EB0EF11C80E4F70111928A9553
:100C7000E9F7D8011896ED91FC91199782818111BD
:100C800003C0EDE0F1E002C0E0E1F1E0808191819C
:100C9000A28189839A83AB8363E0CE0101960E948F
:100CA0009F0C68E070E0C7010E944A0DF80182A520
:100CB000882309F48CC020E4F701C8018E589F4FA7
:100CC000DC0101900D922A95E1F728E0F8013F96AA
:100CD000DF011D922A95E9F7DC0120E030E047E0D2
:100CE00050E06D91F90183E0F595E7958A95E1F77C
:100CF000E00FF11F81E090E0611102C080E090E020
:100D0000B901677077273A01661A770A01C0880F20
:100D10006A94EAF79785892B87872F5F3F4F2034A6
:100D20003105F9F662E571E0F80120E030E0DB0121
:100D30005D91BD01818990E0418D450F841B910932
:100D400047FD939597FD07C08F3F910529F024F04B
:100D50008FEF90E001C080E0818BA8014E575F4F7C
:100D6000982F9078DA019C934F5F5F4F982F907483
:100D7000DA019C934F5F5F4F982F9072DA019C933A
:100D80004F5F5F4F982F9071DA019C934F5F5F4FD9
:100D9000982F9870DA019C934F5F5F4F982F947053
:100DA000DA019C934F5F5F4F982F9270DA019C930A
:100DB0004F5F5F4F8170DA018C932F5F3F4F319609
:100DC000085F1F4F2630310509F0B1CF02C0F8018E
:100DD00011A20F900F900F900F90DF91CF911F9164
:100DE0000F91FF90EF90DF90CF90BF90AF909F90CA
:100DF0008F907F906F9008950C94FE2560E070E0D6
:100E00000C94170CEF92FF920F931F93CF93DF93E5
:100E1000CDB7DEB728970FB6F894DEBF0FBECDBFB3
:100E20008C01FC01E85BFE4F8081909102019F5F85
:100E300090930201833440F4813408F075C0882314
:100E400031F0803421F187C08F3F09F084C0FF2446
:100E5000F394F0928A0289E0F8018383148283E09C
:100E6000858380E886831782108611861286F38632
:100E7000F48640E063E0C80103960E94620BF8012B
:100E8000F4A660E070E0C8010E94170C64C0809175
:100E90008A02882379F0F0908902F9E0FF1554F076
:100EA0006AE070E080E090E00E94C00EF394F0925F
:100EB000890237C0109289028091880298012C5DC6
:100EC0003F4F790181110CC028E0C8010396FC0155
:100ED000D70101900D922A95E1F741E068E00CC03E
:100EE00088E0F901DE01119601900D928A95E1F7F3
:100EF00041E068E0CE0101960E94620BF801EF2804
:100F000011F4128207C0E65BFE4F808181708083FE
:100F1000F801828361E070E0C8010E94170C8093A1
:100F2000880210928A0217C010928A02F801138276
:100F300080E88483858386838783808711861286F1
:100F400081E08387848741E06AE0C80103960E94BC
:100F5000620BF80114A628960FB6F894DEBF0FBEF8
:100F6000CDBFDF91CF911F910F91FF90EF9008952A
:100F7000FC01848DDF01A80FB11DA35ABF4F2C9136
:100F8000848D90E001968F739927848FA689B78905
:100F90002C93A089B1898C91837080648C93938DFC
:100FA000848D981306C00288F389E02D80818F7D9F
:100FB00080830895CF93DF93EC01888D8823C9F057
:100FC000EA89FB89808185FD05C0A889B9898C9152
:100FD00086FD0FC00FB607FCF5CF808185FFF2CFED
:100FE000A889B9898C9185FFEDCFCE010E94B80701
:100FF000E7CFDF91CF910895CF92DF92EF92FF92EA
:101000000F931F93CF93DF93EC011A8280EC91E052
:10101000998388831C821B82198618868FE790E04B
:10102000998B888B1B861A869B8B8A8B1D861C86C8
:101030009D8B8C8B1F861E869F8B8E8B00912B0326
:1010400010912C030115110509F05DC082E00E948A
:1010500040098C0190932C0380932B03009779F522
:1010600069E070E082E00E94B50890932C038093C1
:101070002B03892B09F46BC000E010E080912B0357
:1010800090912C0360E0800F911F0E94F4148091D6
:101090002B0390912C03800F911F6FE701960E9404
:1010A000F4140E5F1F4F0830110541F780912B0398
:1010B00090912C0360E008960E94F41448C00896B2
:1010C0000E94E42290E09C838B837E0188E0E80EFE
:1010D000F11C6E01E0E1CE0ED11CC8010E94E42299
:1010E00090E0F701819391937F01C80101960E94DE
:1010F000E42290E0F701978386830E5F1F4FCE14A2
:10110000DF0459F724C0C80108960E94E42290E049
:101110009C838B837E01F8E0EF0EF11C6E0180E171
:10112000C80ED11CC8010E94E42290E0F70181930F
:1011300091937F01C80101960E94E42290E0F7019B
:10114000978386830E5F1F4FEC14FD0459F781E0EF
:1011500090E09E838D83DF91CF911F910F91FF903F
:10116000EF90DF90CF90089508958F929F92AF9265
:10117000BF92CF92DF92EF92FF920F931F93CF9384
:10118000DF93C82E5B01E0908C02F0908D02C0E0EE
:10119000D0E00AE010E0EC16FD060CF462C0C801D5
:1011A0000E94E42298012E5F3F4F49018F3F21F0BA
:1011B000EC16FD0609F04CC0C4010E94E422D82EB2
:1011C000EC16FD0651F090E08A159B050CF440C02A
:1011D0009C2F8D2FE701E92EF82E6C2DC8010E945F
:1011E000F41460E0C80101960E94F4140D5F1F4FD3
:1011F000EC16FD06A1F08D2D90E00297A816B90619
:101200008CF47801EA0CFB1C6FEFC7010E94F41408
:101210006D2D6A196350C70102960E94F41421963D
:101220006A2D01C06D2DC4010E94F41480918C02BE
:1012300090918D028C179D0749F0D0938D02C09339
:101240008C026C2F81E090E00E94F414C8010BC066
:10125000C4010E94E42290E00396080F191F219612
:101260009ACF80E090E0DF91CF911F910F91FF9096
:10127000EF90DF90CF90BF90AF909F908F900895A8
:10128000DF92EF92FF920F931F93CF93DF93D82EAD
:10129000E0908C02F0908D0200E010E0CAE0D0E017
:1012A0000E151F05CCF4CE010E94E422D81209C00D
:1012B000CE0101960E94E422811103C0CE01039663
:1012C0000DC0CE0102960E94E42290E00396C80F62
:1012D000D91F0F5F1F4FE4CF80E090E0DF91CF91E7
:1012E0001F910F91FF90EF90DF9008950F931F9340
:1012F000CF93DF93EC018B018E819F81009721F0CA
:101300000E94FE251F821E828A819B81009711F018
:101310000E94FE251B830A83DF91CF911F910F91BD
:1013200008950F931F93CF93DF93EC018B018C8172
:101330009D81009711F00E94FE251D830C83DF9193
:10134000CF911F910F9108950F931F93CF93DF9328
:10135000EC01142F022F6230F9F0633069F1613033
:1013600069F085E090E00E946625FC011282D4833A
:10137000C3838EED91E0918380832EC086E090E060
:101380000E946625FC011283D483C38386ED91E01D
:1013900091838083158220C087E090E00E946625BB
:1013A000FC011283D483C38386EC91E09183808314
:1013B00081E0011110C00EC087E090E00E94662518
:1013C000FC011283D483C3838EEC91E091838083EC
:1013D00081E0011180E08683CF01DF91CF911F91E1
:1013E0000F9108952F923F924F925F926F927F924A
:1013F0008F929F92AF92BF92CF92DF92EF92FF9225
:101400000F931F93CF93DF93CDB7DEB728970FB617
:10141000F894DEBF0FBECDBF9E838D836A017B0132
:1014200020E030E040E053E4C701B6010E94C6244A
:10143000181654F420E030E040E853E4C701B60148
:101440000E94FA226B017C0120E030E0A901C70173
:10145000B6010E94672387FF0BC0F7FAF094F7F8F4
:10146000F094812C912C90E8A92E9FEBB92E13C0FB
:1014700020E030E0A901C701B6010E94672388235C
:1014800039F0812C912C80E8A82E8FE3B82E03C070
:10149000812C912C5401ED81FE8127803084B10193
:1014A000032C000C880B990B0E9416242B013C0185
:1014B000A70196010E946723ED81FE8118160CF4A6
:1014C000B5C001851285B801012E000C880B990B5F
:1014D0000E94162469837A838B839C83A7019601DB
:1014E0000E94C62418160CF041C0ED81FE810584CF
:1014F000F685E02DFA83E983ED81FE8163857485AD
:1015000029813A81621B730B072E000C880B990B03
:101510000E9416246D837E838F839887A301920196
:10152000C701B6010E94FA229B01AC016D817E8148
:101530008F8198850E94CB246B017C01B8016219D0
:101540007309072E000C880B990B0E9416249B012F
:10155000AC01C701B6010E946C236B017C01E981DB
:10156000FA81BF01FF0F880B990B40C020E030E0EB
:101570004EEF52E4C701B6010E94672387FF3DC0CA
:10158000ED81FE81238434846FE770E06219730972
:10159000072E000C880B990B0E9416242B013C018E
:1015A00029813A814B815C81C701B6010E94FA22F0
:1015B0009B01AC01C301B2010E94CB246B017C01F1
:1015C0002FE730E0201B310BB901330F880B990B4B
:1015D0000E9416249B01AC01C701B6010E946C2336
:1015E0006B017C01B101330C880B990B0E9416240E
:1015F0009B01AC01C701B60116C020E030E04EEF00
:1016000052E4C701B6010E94FA2220E030E0A901AD
:101610000E94CB2420E030E0A9010E946C2320E04E
:1016200030E04EEF52E40E94FB2210C065857685C3
:10163000072E000C880B990B0E941624A701960117
:101640000E94CB24A30192010E946C23A501940166
:101650000E94CB246B017C0120E030E040E053ECA1
:101660000E94672387FD10C020E030E04EEF52E477
:10167000C701B6010E94C62418164CF0C701B60176
:101680000E94DE23CB0105C080E89FEF02C08FE7F8
:1016900090E028960FB6F894DEBF0FBECDBFDF9165
:1016A000CF911F910F91FF90EF90DF90CF90BF905F
:1016B000AF909F908F907F906F905F904F903F90F2
:1016C0002F900895FC0128E0539A808190E0880FC4
:1016D000892F881F990B892B09F430C00000000066
:1016E000000000000000000000000000539800000F
:1016F00000000000000000000000000000000000EA
:1017000000000000000000000000000000000000D9
:1017100000000000000000000000000000000000C9
:1017200000000000000000000000000000000000B9
:101730000000000000000000000030C000000000B9
:101740000000000000000000000000000000000099
:101750000000000000000000000000000000000089
:101760000000000000000000000000000000000079
:101770000000000000000000000000000000000069
:101780000000000000000000000000000000000059
:10179000000000000000000000005398215069F094
:1017A0000000000000000000000000000000000039
:1017B00000008081880F808387CF00000000000038
:1017C0000000615031F00000000000000000319680
:1017D0007ACF0000000000000000000000000000C0
:1017E0000000539A0000000000000000000000000C
:1017F00000000000000000000000000000000000E9
:101800000000442391F000000000000000000000F0
:1018100000000000000000000000000000000000C8
:101820000000000000000000000053980895CF93CE
:10183000DF93DC01FC01E85BFE4F83E0EF011992CE
:101840008A95E9F7EF01161617069CF484EC99E0E7
:101850004B9907C081E09C968C939C9728E030E0E0
:101860001BC00197A9F79C968C919C97882309F43B
:1018700061C09C968C919C9781110AC080E290E097
:101880004B9902C080E290E0019718161906C4F344
:1018900028E030E04B99FECF00000000000000007F
:1018A0000000000000000000000000000000000038
:1018B0000000000000000000000000000000000028
:1018C0000000000000000000000000000000000018
:1018D0000000000000000000000000000000000008
:1018E000000000004B9B03C08081816080832150F9
:1018F000310931F08081880F80834B9BFECFCACFA6
:101900008881803441F4CD01865B9E4FE817F9074A
:1019100011F03196BDCF4B9BFECF8CE090E04B9900
:1019200002C08CE090E0019718161906C4F381E01C
:1019300090E002C080E090E0DF91CF910895FC013B
:1019400028E08AB180638AB9808190E0880F892F6E
:10195000881F990B892B09F432C000000000000099
:10196000000000000000000000008AB18F7C8AB9EE
:101970000000000000000000000000000000000067
:101980000000000000000000000000000000000057
:101990000000000000000000000000000000000047
:1019A0000000000000000000000000000000000037
:1019B00000000000000000000000000032C0000035
:1019C0000000000000000000000000000000000017
:1019D0000000000000000000000000000000000007
:1019E00000000000000000000000000000000000F7
:1019F00000000000000000000000000000000000E7
:101A000000000000000000000000000000000000D6
:101A10000000000000000000000000008AB18F7C80
:101A20008AB9215069F000000000000000000000A9
:101A300000000000000000008081880F808381CFBB
:101A40000000000000000000615031F000000000C4
:101A500000000000319674CF00000000000000007C
:101A600000000000000000008AB180638AB9000015
:101A70000000000000000000000000000000000066
:101A80000000000000000000000000008AB18F7C10
:101A90008AB90895FC01660F660F660F9FE329B1AE
:101AA000207329F09150D9F780E090E0089500006C
:101AB0000000000000000000000000000000000026
:101AC0000000000000000000000000000000000016
:101AD0000000000000000000000000000000000006
:101AE00000000000000000000000000000000000F6
:101AF0000000000000000000000099B19073919375
:101B0000615051F09FE329B1207309F0C7CF915084
:101B1000D1F782E090E0089581E090E008954F923F
:101B20005F926F927F928F929F92AF92BF92CF926D
:101B3000DF92EF92FF92CF93DF93EC016A017B017A
:101B400020E030E040E053E4C701B6010E94C62423
:101B5000181654F420E030E040E853E4C701B60121
:101B60000E94FA226B017C0120E030E0A901C7014C
:101B7000B6010E94672387FF0BC0F7FAF094F7F8CD
:101B8000F094812C912C40E8A42E4FEBB42E13C07E
:101B900020E030E0A901C701B6010E946723882335
:101BA00039F0812C912C30E8A32E3FE3B32E03C0F3
:101BB000812C912C54018B819C81880F991FC80F17
:101BC000D91F68857985072E000C880B990B0E9418
:101BD00016242B013C01A70196010E94C62487FF11
:101BE00044C0A3019201C701B6010E94FA226B0111
:101BF0007C01A301920160E070E08EEF92E40E940C
:101C0000FA229B01AC01C701B6010E946C236B0153
:101C10007C0168897989072E000C880B990B0E943A
:101C200016249B01AC01C701B6010E94CB24A5017B
:101C300094010E94CB246B017C0120E030E040E065
:101C400053EC0E94672387FD13C020E030E04EEF85
:101C500052E4C701B6010E94C624181664F0C701F9
:101C6000B6010E94DE23CB0108C080E090E005C0F1
:101C700080E89FEF02C08FE790E0DF91CF91FF9067
:101C8000EF90DF90CF90BF90AF909F908F907F901C
:101C90006F905F904F900895CF93DF9390E0FC0199
:101CA000EC55FF4F2491FC01E057FF4F84918823AE
:101CB000C1F090E0880F991FFC01EA57FF4FC591D2
:101CC000D491FC01E458FF4FA591B4919FB7F894CB
:101CD0008881E22FE0958E2388838C91E823EC9312
:101CE0009FBFDF91CF91089590E0FC01E859FF4F2D
:101CF0002491FC01EC55FF4F3491FC01E057FF4F5C
:101D0000E491EE23B9F1222339F1233091F038F434
:101D10002130A9F0223001F584B58F7D12C0273023
:101D200091F02830A1F02430B9F4809180008F7DAB
:101D300003C0809180008F77809380000DC084B5B0
:101D40008F7784BD09C08091B0008F7703C08091E8
:101D5000B0008F7D8093B000F0E0EE0FFF1FE458DD
:101D6000FF4FA591B4919FB7F8948C91309538238B
:101D70003C939FBF0895682F8EE892E00C94C100B9
:101D80008F929F92AF92BF92CF92DF92EF92FF928B
:101D90006B017C010E940E014B015C01C114D10456
:101DA000E104F104F1F00E940E01DC01CB0188197D
:101DB0009909AA09BB09883E9340A105B10570F3B2
:101DC00021E0C21AD108E108F10888EE880E83E00C
:101DD000981EA11CB11CC114D104E104F10419F72F
:101DE000DDCFFF90EF90DF90CF90BF90AF909F90AE
:101DF0008F900895EF92FF920F931F93CF93DF93ED
:101E00008B01EA01E881F981E284F384DB01ED9141
:101E1000FC910084F185E02D61E070E0C801099536
:101E2000482F61E070E0CE01F7010995E881F98162
:101E3000E484F584D801ED91FC910284F385E02DD2
:101E400061E070E0C8010995482F61E070E0CE01C3
:101E5000F7010995E881F981E284F384D801ED91D5
:101E6000FC910084F185E02D62E070E0C8010995E5
:101E7000482F62E070E0CE01F7010995E881F98111
:101E8000E484F584D801ED91FC910284F385E02D82
:101E900062E070E0C8010995482F62E070E0CE0171
:101EA000F7010995E881F981E688F788D801ED9175
:101EB000FC910484F585E02D64E070E0C80109958B
:101EC000482F64E070E0CE01F7010995E881F981BF
:101ED000E688F788D801ED91FC910484F585E02D22
:101EE0006CE070E0C8010995482F6CE070E0CE010D
:101EF000F7010995E881F981E688F788D801ED9125
:101F0000FC910484F585E02D63E070E0C80109953B
:101F1000482F61E070E0CE01F7010995E881F98171
:101F2000E688F788D801ED91FC910484F585E02DD1
:101F300061E070E0C8010995482F62E070E0CE01D1
:101F4000F7010995E881F981E688F788D801ED91D4
:101F5000FC910484F585E02D62E070E0C8010995EC
:101F6000482F63E070E0CE01F7010995E881F9811F
:101F7000E688F788D801ED91FC910484F585E02D81
:101F800060E070E0C8010995482F60E070E0CE0184
:101F9000F7010995E881F981E688F788D801ED9184
:101FA000FC910484F585E02D6DE070E0C801099591
:101FB000482F6DE070E0CE01F7010995E881F981C5
:101FC000E688F788D801ED91FC910484F585E02D31
:101FD0006EE070E0C8010995482F6EE070E0CE0118
:101FE000F7010995E881F981E688F788D801ED9134
:101FF000FC910484F585E02D6BE070E0C801099543
:10200000482F6BE070E0CE01F7010995E881F98176
:10201000E688F788D801ED91FC910484F585E02DE0
:102020006AE070E0C8010995482F6AE070E0CE01CF
:10203000F7010995E881F981E688F788D801ED91E3
:10204000FC910484F585E02D68E070E0C8010995F5
:10205000482F68E070E0CE01F7010995E881F98129
:10206000E688F788D801ED91FC910484F585E02D90
:1020700069E070E0C8010995482F69E070E0CE0181
:10208000F701DF91CF911F910F91FF90EF9009948D
:10209000EF92FF920F931F93CF93DF938B01EA018F
:1020A000E881F981E284F384DB01ED91FC91008405
:1020B000F185E02D61E070E0C8010995482F61E0ED
:1020C00070E0CE01F7010995E881F981E484F58497
:1020D000D801ED91FC910284F385E02D61E070E080
:1020E000C8010995482F61E070E0CE01F70109951C
:1020F000E881F981E284F384D801ED91FC910084B8
:10210000F185E02D62E070E0C8010995482F62E09A
:1021100070E0CE01F7010995E881F981E484F58446
:10212000D801ED91FC910284F385E02D62E070E02E
:10213000C8010995482F62E070E0CE01F7010995CA
:10214000E881F981E688F788D801ED91FC91048453
:10215000F585E02D64E070E0C8010995482F64E042
:1021600070E0CE01F7010995E881F981E688F788EA
:10217000D801ED91FC910484F585E02D6CE070E0D0
:10218000C8010995482F6CE070E0CE01F701099570
:10219000E881F981E688F788D801ED91FC91048403
:1021A000F585E02D60E070E0C8010995482F61E0F9
:1021B00070E0CE01F7010995E881F981E688F7889A
:1021C000D801ED91FC910484F585E02D63E070E089
:1021D000C8010995482F62E070E0CE01F70109952A
:1021E000E881F981E688F788D801ED91FC910484B3
:1021F000F585E02D61E070E0C8010995482F63E0A6
:1022000070E0CE01F7010995E881F981E688F78849
:10221000D801ED91FC910484F585E02D62E070E039
:10222000C8010995482F60E070E0CE01F7010995DB
:10223000E881F981E688F788D801ED91FC91048462
:10224000F585E02D6DE070E0C8010995482F6DE03F
:1022500070E0CE01F7010995E881F981E688F788F9
:10226000D801ED91FC910484F585E02D6EE070E0DD
:10227000C8010995482F6EE070E0CE01F70109957D
:10228000E881F981E688F788D801ED91FC91048412
:10229000F585E02D6BE070E0C8010995482F6BE0F3
:1022A00070E0CE01F7010995E881F981E688F788A9
:1022B000D801ED91FC910484F585E02D6AE070E091
:1022C000C8010995482F6AE070E0CE01F701099531
:1022D000E881F981E688F788D801ED91FC910484C2
:1022E000F585E02D68E070E0C8010995482F68E0A9
:1022F00070E0CE01F7010995E881F981E688F78859
:10230000D801ED91FC910484F585E02D69E070E041
:10231000C8010995482F69E070E0CE01F701DF910F
:10232000CF911F910F91FF90EF900994EF92FF9240
:102330000F931F93CF93DF938B01EA01E881F9811B
:10234000E284F384DB01ED91FC910084F185E02DC2
:1023500061E070E0C8010995482F61E070E0CE01AE
:10236000F7010995E881F981E484F584D801ED91BC
:10237000FC910284F385E02D61E070E0C8010995CD
:10238000482F61E070E0CE01F7010995E881F981FD
:10239000E284F384D801ED91FC910084F185E02D75
:1023A00062E070E0C8010995482F62E070E0CE015C
:1023B000F7010995E881F981E484F584D801ED916C
:1023C000FC910284F385E02D62E070E0C80109957C
:1023D000482F62E070E0CE01F7010995E881F981AC
:1023E000E688F788D801ED91FC910484F585E02D0D
:1023F00064E070E0C8010995482F64E070E0CE0108
:10240000F7010995E881F981E688F788D801ED910F
:10241000FC910484F585E02D6CE070E0C80109951D
:10242000482F6CE070E0CE01F7010995E881F98151
:10243000E688F788D801ED91FC910484F585E02DBC
:1024400061E070E0C8010995482F61E070E0CE01BD
:10245000F7010995E881F981E688F788D801ED91BF
:10246000FC910484F585E02D62E070E0C8010995D7
:10247000482F62E070E0CE01F7010995E881F9810B
:10248000E688F788D801ED91FC910484F585E02D6C
:1024900063E070E0C8010995482F63E070E0CE0169
:1024A000F7010995E881F981E688F788D801ED916F
:1024B000FC910484F585E02D60E070E0C801099589
:1024C000482F60E070E0CE01F7010995E881F981BD
:1024D000E688F788D801ED91FC910484F585E02D1C
:1024E0006DE070E0C8010995482F6DE070E0CE0105
:1024F000F7010995E881F981E688F788D801ED911F
:10250000FC910484F585E02D6EE070E0C80109952A
:10251000482F6EE070E0CE01F7010995E881F9815E
:10252000E688F788D801ED91FC910484F585E02DCB
:102530006BE070E0C8010995482F6BE070E0CE01B8
:10254000F7010995E881F981E688F788D801ED91CE
:10255000FC910484F585E02D6AE070E0C8010995DE
:10256000482F6AE070E0CE01F7010995E881F98112
:10257000E688F788D801ED91FC910484F585E02D7B
:1025800068E070E0C8010995482F68E070E0CE016E
:10259000F7010995E881F981E688F788D801ED917E
:1025A000FC910484F585E02D69E070E0C80109958F
:1025B000482F69E070E0CE01F701DF91CF911F91C4
:1025C0000F91FF90EF900994EF92FF920F931F935A
:1025D000CF93DF938B01EA01E881F981E284F384F0
:1025E000DB01ED91FC910084F185E02D60E070E06D
:1025F000C8010995482F60E070E0CE01F701099508
:10260000E881F981E484F584D801ED91FC9102849C
:10261000F385E02D60E070E0C8010995482F60E087
:1026200070E0CE01F701DF91CF911F910F91FF90E4
:10263000EF9009944F925F926F927F92AF92BF9208
:10264000CF92DF92EF92FF920F931F93CF93DF937E
:10265000EB018A01DA01ED91FC91E284F384E881D7
:10266000F9810084F185E02D61E070E0CE010995EB
:10267000482F61E070E0C801F7010995D801ED919C
:10268000FC91E484F584E881F9810284F385E02DEE
:1026900061E070E0CE010995482F61E070E0C8016B
:1026A000F7010995E881F9810084F185E02D62E068
:1026B00070E0CE010995682F880F770B60587F4F27
:1026C000072E000C880B990B0E94162420E030E0A6
:1026D00045E553E40E94CB2420E030E044E752E497
:1026E0000E946C236B017C01E881F9810284F385EF
:1026F000E02D62E070E0CE010995682F880F770B1E
:1027000060587F4F072E000C880B990B0E941624EF
:1027100020E030E045E553E40E94CB2420E030E0A7
:1027200044E752E40E946C232B013C01D801ED9157
:10273000FC91A284B38420E030E04FE753E4C7016A
:10274000B6010E94C624181664F020E030E040E094
:1027500053E4C701B6010E94FA220E94DE23462FED
:1027600001C04FE762E070E0C801F5010995D801AA
:10277000ED91FC91E484F58420E030E04FE753E4F0
:10278000C301B2010E94C624181664F020E030E0B4
:1027900040E053E4C301B2010E94FA220E94DE230A
:1027A000462F01C04FE762E070E0C801F7010995CC
:1027B000D801ED91FC91E688F788E881F9810484DD
:1027C000F585E02D64E070E0CE010995482F64E0C6
:1027D00070E0C801F7010995D801ED91FC91E688F8
:1027E000F788E881F9810484F585E02D6CE070E0DC
:1027F000CE010995482F6CE070E0C801F7010995FA
:10280000D801ED91FC91E688F788E881F98104848C
:10281000F585E02D61E070E0CE010995482F61E07B
:1028200070E0C801F7010995D801ED91FC91E688A7
:10283000F788E881F9810484F585E02D62E070E095
:10284000CE010995482F62E070E0C801F7010995B3
:10285000D801ED91FC91E688F788E881F98104843C
:10286000F585E02D63E070E0CE010995482F63E027
:1028700070E0C801F7010995D801ED91FC91E68857
:10288000F788E881F9810484F585E02D60E070E047
:10289000CE010995482F60E070E0C801F701099565
:1028A000D801ED91FC91E688F788E881F9810284EE
:1028B000F385E02D62E070E0CE010995D82EE88125
:1028C000F9810484F585E02D6DE070E0CE01099575
:1028D00041E0BDEBDB160CF440E0482B6DE070E00E
:1028E000C801F7010995D801ED91FC91E688F788B8
:1028F000E881F9810084F185E02D62E070E0CE018D
:102900000995D82EE881F9810484F585E02D6EE0E3
:1029100070E0CE01099541E0BDEBDB160CF440E020
:10292000482B6EE070E0C801F7010995D801ED91E0
:10293000FC91E688F788E881F9810484F585E02D2B
:102940006BE070E0CE010995482F6BE070E0C801A4
:10295000F7010995D801ED91FC91E688F788E881A7
:10296000F9810484F585E02D6AE070E0CE010995D7
:10297000482F6AE070E0C801F7010995D801ED9190
:10298000FC91E688F788E881F9810484F585E02DDB
:1029900068E070E0CE010995482F68E070E0C8015A
:1029A000F7010995D801ED91FC91E688F788E88157
:1029B000F9810484F585E02D69E070E0CE01099588
:1029C000482F69E070E0C801F701DF91CF911F91B6
:1029D0000F91FF90EF90DF90CF90BF90AF907F90DE
:1029E0006F905F904F9009940F931F93CF938C013A
:1029F000C62F0E94E422C81721F06C2FC8010E9444
:102A0000EC228C2FCF911F910F910895CF92DF92DE
:102A1000FF920F931F93CF93DF938C01EA01E8811C
:102A2000F981C284D384DC011796ED91FC9118974B
:102A300082859385DC01ED91FC910190F081E02D80
:102A40000995F82ED8011796ED91FC91189780857D
:102A50009185DC01ED91FC910190F081E02D0995CB
:102A6000F69486954F2D481B61E070E0CE01F6018B
:102A70000995E881F981C484D584D8011796ED9130
:102A8000FC91189786859785DC01ED91FC9101906A
:102A9000F081E02D0995F82ED8011796ED91FC9163
:102AA000189784859585DC01ED91FC910190F0816A
:102AB000E02D0995F69486954F2D481B61E070E056
:102AC000CE01F6010995E881F981C284D384D80149
:102AD0001796ED91FC91189780899189DC01ED9111
:102AE000FC910190F081E02D0995482F62E070E0A3
:102AF000CE01F6010995E881F981C484D584D80115
:102B00001796ED91FC91189782899389DC01ED91DC
:102B1000FC910190F081E02D0995482F62E070E072
:102B2000CE01F6010995E881F981C688D788D801D8
:102B30001796ED91FC91189784899589DC01ED91A8
:102B4000FC910280F381E02D099541E0811101C0E3
:102B500040E060E070E0CE01F6010995E881F9817E
:102B6000C688D788D8011796ED91FC911897868969
:102B70009789DC01ED91FC910280F381E02D0995AC
:102B800041E0811101C040E061E070E0CE01F6015A
:102B90000995E881F981C688D788D8011796ED9103
:102BA000FC911897808D918DDC01ED91FC91028054
:102BB000F381E02D099541E0811101C040E062E020
:102BC00070E0CE01F6010995E881F981C688D788C1
:102BD000D8011796ED91FC911897828D938DDC01A9
:102BE000ED91FC910280F381E02D099541E0811186
:102BF00001C040E063E070E0CE01F6010995E88194
:102C0000F981C688D788D8011796ED91FC9118975D
:102C1000848D958DDC01ED91FC910280F381E02D96
:102C2000099541E0811101C040E064E070E0CE010F
:102C3000F6010995E881F981C688D788D8011796E9
:102C4000ED91FC911897868D978DDC01ED91FC91AB
:102C50000280F381E02D099541E0811101C040E03F
:102C600068E070E0CE01F6010995E881F981C68837
:102C7000D788D8011796ED91FC91189780A191A162
:102C8000DC01ED91FC910280F381E02D099541E09A
:102C9000811101C040E069E070E0CE01F6010995C4
:102CA000E881F981C688D788D8011796ED91FC9103
:102CB000189782A193A1DC01ED91FC910280F38130
:102CC000E02D099541E0811101C040E06AE070E02B
:102CD000CE01F6010995E881F981C688D788D80127
:102CE0001796ED91FC91189784A195A1DC01ED91C7
:102CF000FC910280F381E02D099541E0811101C032
:102D000040E06BE070E0CE01F6010995E881F981C1
:102D1000C688D788D8011796ED91FC91189786A19F
:102D200097A1DC01ED91FC910280F381E02D0995E2
:102D300041E0811101C040E06CE070E0CE01F6019D
:102D40000995E881F981C688D788D8011796ED9151
:102D5000FC91189780A591A5DC01ED91FC91028072
:102D6000F381E02D099541E0811101C040E06DE063
:102D700070E0CE01F6010995E881F981C688D7880F
:102D8000D8011796ED91FC91189782A593A5DC01C7
:102D9000ED91FC910280F381E02D099541E08111D4
:102DA00001C040E06EE070E0CE01F601DF91CF910E
:102DB0001F910F91FF90DF90CF900994CF93DF93F5
:102DC000FC018681A381B4816281882369F0062E8B
:102DD000000C770BED91FC9111970680F781E02DA7
:102DE000CD01DF91CF910994EF01062E000C770BF6
:102DF000ED91FC9111970680F781E02DCD010995A9
:102E00002FEF30E0A901481B51092D8130E02058F7
:102E10003F4F81E0241735070CF480E0DF91CF911C
:102E200008958F929F92AF92BF92CF92DF92EF92CE
:102E3000FF92CF93DF93EC012E818B819C816A817D
:102E4000062E000C770BDC01ED91FC910680F781DA
:102E5000E02D222311F0099502C0099580959D81EE
:102E6000E92EF12C282F30E0A70140585F4F421780
:102E700053070CF04CC0682F691B605870E080E06D
:102E800090E00E9414244B015C016FE770E06E1922
:102E90007F09072E000C880B990B0E9416249B01BA
:102EA000AC01C501B4010E946C2320E030E04FE783
:102EB00053E40E94CB246B017C0120E030E0A901A7
:102EC0000E94672318161CF520E030E04FE753E41A
:102ED000C701B6010E94C62487FF1BC020E030E076
:102EE000A901C701B6010E94C62420E030E040E0FD
:102EF0005FE387FD05C0C701B6010E94FB2204C045
:102F0000C701B6010E94FA220E94DE2303C060E0DE
:102F100001C06FEF862FDF91CF91FF90EF90DF9090
:102F2000CF90BF90AF909F908F900895CF93DF93F5
:102F3000EC012E818B819C816A81062E000C770B1F
:102F4000DC01ED91FC910680F781E02D222331F028
:102F500009952FEF30E0281B310903C00995282F70
:102F600030E04D8150E081E0241735070CF480E01B
:102F7000DF91CF9108958F929F92AF92BF92CF929F
:102F8000DF92EF92FF92CF93DF93EC012E818B8142
:102F90009C816A81062E000C770BDC01ED91FC917F
:102FA0000680F781E02D222319F00995809501C054
:102FB0000995682F880F770BED80F12C6E157F0532
:102FC0000CF44CC06E197F09072E000C880B990B6E
:102FD0000E9416244B015C016FEF70E06E197F09AF
:102FE000072E000C880B990B0E9416249B01AC0144
:102FF000C501B4010E946C2320E030E04FE753E4A8
:103000000E94CB246B017C0120E030E0A9010E94EA
:10301000672318161CF520E030E04FE753E4C701A2
:10302000B6010E94C62487FF1BC020E030E0A90142
:10303000C701B6010E94C62420E030E040E05FE313
:1030400087FD05C0C701B6010E94FB2204C0C7016D
:10305000B6010E94FA220E94DE2303C060E001C094
:103060006FEF862FDF91CF91FF90EF90DF90CF90A1
:10307000BF90AF909F908F900895CF93DF93EC0116
:103080008B819C816A81062E000C770BDC01ED910F
:10309000FC910484F585E02D0995882311F08D813C
:1030A00001C080E0DF91CF910895FC01A381B4813C
:1030B0006281062E000C770BED91FC911197048430
:1030C000F585E02DCD01099480E0089520912F032E
:1030D000309130032115310529F0682FC90101967F
:1030E0000C94F4140895682F80912F03909130036D
:1030F000009711F00C94F41408950F931F93CF933D
:10310000DF938C0186E791E0F8019183808382E868
:1031100091E093838283C0E0D0E0F801258136817D
:1031200087819085C217D30764F49E01220F331F55
:10313000FC01E20FF31F808191810E94FE25219600
:10314000ECCF009731F0DF91CF911F910F910C944C
:10315000FE25DF91CF911F910F91089580912F034C
:1031600090913003892BF9F480E00E9440099093FC
:10317000300380932F03892BB1F462E070E080E08C
:103180000E94B5089093300380932F03009759F065
:1031900061E00E94F41480912F039091300360E06D
:1031A00001960C94F41408950F931F93CF93DF931B
:1031B0008C01EB01FC018381E881F981882359F0BE
:1031C0000088F189E02DCB010995882309F4F6C028
:1031D000F8011382F3C00484F585E02D64E070E00B
:1031E000CE010995882381F083E090E00E94662556
:1031F000FC01128226EA31E031832083BC01CE013A
:103200000E94760980E017C0E881F9810484F58581
:10321000E02D61E070E0CE010995882391F081E115
:1032200090E00E9466258C010E94681DB801CE01C5
:103230000E94760981E0DF91CF911F910F910C944C
:103240007318E881F9810484F585E02D6EE070E063
:10325000CE0109958823A9F082E090E00E946625BE
:1032600020EA31E0FC0131832083BC01CE010E94C1
:1032700091098E819F819B838A831F821E8280E0B9
:1032800097C0E881F9810484F585E02D63E070E062
:10329000CE010995882369F088E190E00E946625B7
:1032A0008C010E94FC07B801CE010E94760982E0E1
:1032B000C2CFE881F9810484F585E02D69E070E0F2
:1032C000CE0109958823A9F082E090E00E9466254E
:1032D0002AE931E0FC0131832083BC01CE010E9448
:1032E00091098E819F819B838A831F821E8281E048
:1032F0005FC0E881F9810484F585E02D68E070E025
:10330000CE0109958823A9F082E090E00E9466250D
:1033100028E831E0FC0131832083BC01CE010E940A
:1033200091098E819F819B838A831F821E8284E004
:103330003FC0E881F9810484F585E02D6AE070E002
:10334000CE0109958823A9F082E090E00E946625CD
:1033500024E931E0FC0131832083BC01CE010E94CD
:1033600091098E819F819B838A831F821E8282E0C6
:103370001FC0E881F9810484F585E02D6BE070E0E1
:10338000CE0109958823D1F082E090E00E94662565
:103390002EE831E0FC0131832083BC01CE010E9484
:1033A00091098E819F819B838A831F821E8283E085
:1033B000DF91CF911F910F910C946618DF91CF91FF
:1033C0001F910F910895EF92FF920F931F93CF9348
:1033D000DF938B01EA01E881F981E284F384DB0168
:1033E000ED91FC910084F185E02D61E070E0C80171
:1033F0000995482F61E070E0CE01F7010995E88159
:10340000F981E484F584D801ED91FC910284F3857F
:10341000E02D61E070E0C8010995482F61E070E09F
:10342000CE01F7010995E881F981E284F384D8019E
:10343000ED91FC910484F585E02D6EE070E0C8010B
:103440000995811102C042E801C04FE762E070E0D7
:10345000CE01F7010995E881F981E484F584D8016A
:10346000ED91FC910484F585E02D6DE070E0C801DC
:103470000995811102C042E801C04FE762E070E0A7
:10348000CE01F7010995E881F981E688F788D8012E
:10349000ED91FC910484F585E02D64E070E0C801B5
:1034A0000995482F64E070E0CE01F7010995E881A5
:1034B000F981E688F788D801ED91FC910484F585BF
:1034C000E02D6CE070E0C8010995482F6CE070E0D9
:1034D000CE01F7010995E881F981E688F788D801DE
:1034E000ED91FC910484F585E02D61E070E0C80168
:1034F0000995482F61E070E0CE01F7010995E88158
:10350000F981E688F788D801ED91FC910484F5856E
:10351000E02D62E070E0C8010995482F62E070E09C
:10352000CE01F7010995E881F981E688F788D8018D
:10353000ED91FC910484F585E02D63E070E0C80115
:103540000995482F63E070E0CE01F7010995E88105
:10355000F981E688F788D801ED91FC910484F5851E
:10356000E02D60E070E0C8010995482F60E070E050
:10357000CE01F7010995E881F981E688F788D8013D
:10358000ED91FC910484F585E02D6DE070E0C801BB
:103590000995482F6DE070E0CE01F7010995E881AB
:1035A000F981E688F788D801ED91FC910484F585CE
:1035B000E02D6EE070E0C8010995482F6EE070E0E4
:1035C000CE01F7010995E881F981E688F788D801ED
:1035D000ED91FC910484F585E02D6BE070E0C8016D
:1035E0000995482F6BE070E0CE01F7010995E8815D
:1035F000F981E688F788D801ED91FC910484F5857E
:10360000E02D6AE070E0C8010995482F6AE070E09B
:10361000CE01F7010995E881F981E688F788D8019C
:10362000ED91FC910484F585E02D68E070E0C8011F
:103630000995482F68E070E0CE01F7010995E8810F
:10364000F981E688F788D801ED91FC910484F5852D
:10365000E02D69E070E0C8010995482F69E070E04D
:10366000CE01F701DF91CF911F910F91FF90EF9065
:103670000994DF92EF92FF920F931F93CF93DF9302
:10368000EC018B017A018C819D818130910521F0C3
:10369000029709F471C011C0DB01ED91FC91028821
:1036A000F389E02DCB010995882329F082E090E091
:1036B0009D838C83DDC11D821C82D801ED91FC911C
:1036C0000084F185E02D60E070E0C8010995D80123
:1036D000ED91FC910284F385E02D60E070E0C8017B
:1036E0000995D801ED91FC910084F185E02D60E011
:1036F00070E0C8010995682F880F770B880B990B2C
:103700000E941624AB01BC01CE010E94F209D82E02
:10371000D801ED91FC910284F385E02D60E070E02A
:10372000C8010995682F880F770B880B990B0E94A9
:103730001624AB01BC01CE010E94F209C82FD701AB
:10374000ED91FC910284F385E02D4D2D60E070E059
:10375000C7010995D701ED91FC910484F585E02D11
:103760004C2F60E070E0C701DF91CF911F910F9166
:10377000FF90EF90DF900994AF81B885A650BE4FBF
:10378000FA0180819181FC01228533854C9160E0B2
:1037900070E0C701F9010995A985BA85A650BE4F09
:1037A000F70180819181FC01248535854C9160E091
:1037B00070E0C701F9010995D801ED91FC910288EB
:1037C000F389E02DC8010995882309F454C18E813D
:1037D000D801ED91FC910484F585E02D882309F44E
:1037E00068C062E070E0C801099581115FC1D8012D
:1037F000ED91FC910484F585E02D63E070E0C80153
:103800000995811153C1D801ED91FC910484F5858E
:10381000E02D61E070E0C8010995811147C1D80130
:10382000ED91FC910484F585E02D60E070E0C80125
:10383000099581113BC1D801ED91FC910484F58576
:10384000E02D68E070E0C801099581112FC1D80111
:10385000ED91FC910484F585E02D69E070E0C801EC
:103860000995811123C1D801ED91FC910484F5855E
:10387000E02D6AE070E0C8010995811117C1D801F7
:10388000ED91FC910484F585E02D6CE070E0C801B9
:10389000099581110BC1D801ED91FC910484F58546
:1038A000E02D64E070E0C80109958111FFC01E821F
:1038B000FDC063E070E0C8010995882351F08F8155
:1038C00098858230910514F0019719C081E090E04D
:1038D00016C0D801ED91FC910484F585E02D62E0DD
:1038E00070E0C8010995882369F02F8138858985A2
:1038F0009A8501972817390714F4C901019698870A
:103900008F83B6C0D801ED91FC910484F585E02D3C
:1039100061E070E0C8010995882361F029853A8546
:103920008F8198850196821793070CF051C0C901C9
:1039300001974EC0D801ED91FC910484F585E02DEE
:1039400060E070E0C8010995882351F089859A8567
:103950008E37910514F401963BC08EE790E038C095
:10396000D801ED91FC910484F585E02D64E070E0D0
:10397000C80109958823D1F08B81813049F08230CC
:1039800071F087E190E098878F8385E290E020C016
:1039900084E190E098878F8380E290E019C08EE107
:1039A00090E098878F8389E290E012C0D801ED9172
:1039B000FC910484F585E02D6CE070E0C801099568
:1039C000882349F088E090E098878F838AE290E02E
:1039D0009A8789874DC0D801ED91FC910484F585C3
:1039E000E02D68E070E0C8010995882369F082E065
:1039F0008B838EE190E09E878D8789E290E09C87A3
:103A00008B8789E490E032C0D801ED91FC91048469
:103A1000F585E02D6AE070E0C8010995882379F00A
:103A200081E08B8324E130E03E872D8720E230E087
:103A30003C872B8725E330E0388B2F871AC0D801CD
:103A4000ED91FC910484F585E02D69E070E0C801FA
:103A50000995882359F11B8287E190E09E878D8725
:103A600085E290E09C878B8787E490E0988B8F8736
:103A700081E08E831BC080912D0390912E030097CF
:103A800099F06F810E94F41480912D0390912E0380
:103A9000698501960E94F41480912D0390912E0364
:103AA0006B8102960E94F4141D821C82DF91CF91DB
:103AB0001F910F91FF90EF90DF900895CF93DF93C8
:103AC000EC010E947D18CE01DF91CF910C94FE2570
:103AD0000F931F93CF93DF93EC011A8288EF91E04D
:103AE000998388831B8200912D0310912E03011569
:103AF0001105F1F581E00E9440098C0190932E039D
:103B000080932D03892BA1F563E070E081E00E9492
:103B1000B50890932E0380932D031B8227E130E09C
:103B20003E872D8725E230E03C872B8727E430E075
:103B3000388B2F8728E030E038872F832AE230E067
:103B40003A872987009731F168E00E94F414809148
:103B50002D0390912E03698501960E94F4148091A3
:103B60002D0390912E036B8102960E94F41412C0D3
:103B7000C8010E94E42290E098878F83C8010196D3
:103B80000E94E42290E09A878987C80102960E94E9
:103B9000E4228B838B81813069F08230B1F087E140
:103BA00090E09E878D8785E290E09C878B8787E4F5
:103BB00090E015C084E190E09E878D8780E290E0E0
:103BC0009C878B8785E390E00AC08EE190E09E871A
:103BD0008D8789E290E09C878B8789E490E0988BC1
:103BE0008F8789859A858038910524F08EE790E04B
:103BF0009A87898789859A852F81388582179307C7
:103C00001CF4019798878F8381E090E09D838C83DB
:103C1000DF91CF911F910F910895CF93DF9300D043
:103C200000D000D0CDB7DEB7789484B5826084BD73
:103C300084B5816084BD85B5826085BD85B58160B0
:103C400085BD80916E00816080936E00109281002E
:103C500080918100826080938100809181008160E9
:103C600080938100809180008160809380008091AA
:103C7000B10084608093B1008091B0008160809336
:103C8000B00080917A00846080937A0080917A00FD
:103C9000826080937A0080917A00816080937A00BC
:103CA00080917A00806880937A001092C100E09140
:103CB0009E02F0919F0282E08083E0919A02F0914F
:103CC0009B021082E0919C02F0919D0280E1808332
:103CD0001092A602E091A202F091A30286E08083F6
:103CE000E091A002F091A102808180618083E09147
:103CF000A002F091A102808188608083E091A002FF
:103D0000F091A102808180688083E091A002F0910F
:103D1000A10280818F7D80838091000190910101BB
:103D20000197909301018093000143E050E062E02D
:103D300070E0CE0104960E94D4228C81853A31F441
:103D40008D818E3919F48E818C3811F080E052C04B
:103D500060E085E090E00E94F41489E090E00E9429
:103D6000E4228233A1F162E389E090E00E94F4143E
:103D700010928D0210928C0260E080E090E00E9430
:103D8000F41460918C0281E090E00E94F414809120
:103D9000190190911A01A0911B0189839A83AB8329
:103DA000CE0101967C0102E010E0D701DD907D019B
:103DB000C8010E94E422D81621F06D2DC8010E948E
:103DC000EC220F5F1F4F0530110579F712C080E01C
:103DD00090E00E94E42290E090938D0280938C0208
:103DE00081E090E00E94E42290E090938D02809325
:103DF0008C0281E080937E028BE491E00E94662534
:103E00007C0180E291E0F70191838083339681E227
:103E1000DF011D928A95E9F7EB5BFE4F83E0DF013E
:103E20001D928A95E9F7F70114A6F0927D02E092BF
:103E30007C028CEB90E00E9466258C018EE591E07F
:103E4000D80111969C938E93C8018E589F4F1D9652
:103E50009C938E931C9780E490E01B969C938E938A
:103E60001A971E961C921E9791961C9291978AE023
:103E7000E0E5F1E0579601900D928A95E1F71093F5
:103E80007B0200937A0283E00E94740E83E00E941A
:103E90004C0EF701128289E090E00E9466257C01B9
:103EA000DC0114961C92149786E791E011969C937E
:103EB0008E9382E891E013969C938E93129786E1FD
:103EC00090E016969C938E9315978CE290E00E945A
:103ED00066256C01F7019087878321E040E063E06D
:103EE000C8010E94A409D6018D939C93F701C78055
:103EF000D08420E040E063E0C8010E94A409D6011C
:103F000013969C938E931297F701C780D08421E07B
:103F100041E063E0C8010E94A409D60115969C9374
:103F20008E931497F701C780D08420E041E063E0CE
:103F3000C8010E94A409D60117969C938E931697E8
:103F4000F701C780D08421E042E063E0C8010E940D
:103F5000A409D60119969C938E931897F701C780F0
:103F6000D08420E042E063E0C8010E94A409D601A9
:103F70001B969C938E931A97F701C780D08421E0FB
:103F800043E063E0C8010E94A409D6011D969C93FA
:103F90008E931C97F701C780D08420E043E063E054
:103FA000C8010E94A409D6011F969C938E931E9768
:103FB000F701C780D08421E044E062E0C8010E949C
:103FC000A409D60151969C938E935097F701C78010
:103FD000D08421E045E062E0C8010E94A409D60136
:103FE00053969C938E935297F701C780D08420E01C
:103FF00040E061E0C8010E94A409D60155969C9357
:104000008E935497F701C780D08420E041E061E0AF
:10401000C8010E94A409D60157969C938E93569787
:10402000F701C780D08420E042E061E0C8010E942F
:10403000A409D60159969C938E935897F701C7808F
:10404000D08420E043E061E0C8010E94A409D601C9
:104050005B969C938E935A97F701C780D08420E09B
:1040600044E061E0C8010E94A409D6015D969C93DA
:104070008E935C97F701C780D08420E048E061E030
:10408000C8010E94A409D6015F969C938E935E9707
:10409000F701C780D08420E049E061E0C8010E94B8
:1040A000A409D60191969C938E939097F701C780AF
:1040B000D08420E04AE061E0C8010E94A409D60152
:1040C00093969C938E939297F701C780D08420E0BB
:1040D0004BE061E0C8010E94A409D60195969C932B
:1040E0008E939497F701C780D08420E04CE061E084
:1040F000C8010E94A409D60197969C938E93969727
:10410000F701C780D08420E04DE061E0C8010E9443
:10411000A409D60199969C938E939897F701E7800E
:10412000F08420E04EE061E0C8010E94A409D701BC
:104130009B969C938E939A970E94AE1880912F0322
:1041400090913003009769F001960E94E42282303A
:10415000B1F018F4813061F004C08330B9F08430DC
:10416000F9F082E090E00E94662520EA31E01EC06E
:1041700082E090E00E9466252AE931E00DC082E0ED
:1041800090E00E94662524E931E010C082E090E0D2
:104190000E9466252EE831E0DC012D933C9309C096
:1041A00082E090E00E94662528E831E0FC0131833E
:1041B00020836C010E94AE1880912F0390913003F0
:1041C000009731F00E94E422813081F08230B1F01A
:1041D00083E090E00E946625DC0112961C92129703
:1041E00026EA31E02D933C938C010FC081E190E0F1
:1041F0000E9466258C010E94681D07C088E190E03E
:104200000E9466258C010E94FC07A0907C02B09061
:104210007D02E0907A02F0907B0285E00E94740EAD
:1042200085E00E944C0E84E00E94740E84E00E949F
:104230004C0EF701B186A08602831383C482D58217
:10424000178216823CEA632E31E0732E5524539474
:1042500048E0842E912C80917E02882309F4F7C0D7
:1042600080917C0290917D02DC01ED91FC910190A6
:10427000F081E02D09958111D2C000917A02109150
:104280007B02F8018685C484D584A284B384882304
:1042900051F1E12CF12CEA14FB0464F5C701F7FCA1
:1042A000079623E0959587952A95E1F7F601E80FA3
:1042B000F91F2081022E000C330BC701B4010E94AC
:1042C000382502C0359527958A95E2F7C901817096
:1042D000992720FF02C081E390E00E94BB0EFFEF10
:1042E000EF1AFF0AD8CF7601C7018C199D098A15EC
:1042F0009B057CF08AE090E00E94BB0ED801ED9116
:10430000FC910684F785E02DC801099581110EC046
:1043100038C0F70181917F01882319F081E390E093
:1043200002C080E090E00E94BB0EDECFD801129662
:10433000ED91FC911397309719F08281811121C082
:1043400084E090E00E9466257C01FC01718260821D
:1043500053825282892B09F47DC0F80186819781AE
:10436000009711F00E94FE25D80112968D919C9124
:10437000139717969C938E9316971396FC92EE9232
:1043800012976091000170910101072E000C880BBB
:10439000990B0E94C00EF89400917A0210917B0252
:1043A000D801ED91FC910480F581E02DC8010995BB
:1043B000F80180859185DC01ED91FC910084F18507
:1043C000E02D0995F80182819381009751F0408595
:1043D0005185DC01ED91FC910190F081E02DB80157
:1043E0000995F80186819781892B71F484819581E3
:1043F000009751F040855185DC01ED91FC910190D1
:10440000F081E02DB801099580917C0290917D02A8
:10441000DC01ED91FC910480F581E02D09958091FE
:104420007C0290917D02DC01ED91FC910280F38190
:10443000E02D0995F89480917C0290917D02DC0139
:10444000ED91FC910680F781E02D099578940E940A
:10445000120201CFF80186819781938382831782AC
:1044600016828FCFEEE8F2E01382128288EE93E09C
:10447000A0E0B0E084839583A683B78386EE91E0C5
:104480009183808385EC90E09587848784EC90E02D
:104490009787868780EC90E0918B808B81EC90E011
:1044A000938B828B82EC90E0958B848B86EC90E0F2
:1044B000978B868B118E128E138E148E10922C0376
:1044C00010922B0310922E0310922D0310923003A2
:1044D00010922F030895CF92DF92EF92FF920F93E5
:1044E0001F93CF937C018A01DA01ED91FC91C28484
:1044F000D384DC011796ED91FC911897828193810A
:10450000DC01ED91FC910190F081E02D0995C82F1F
:10451000D7011796ED91FC91189780819181DC016C
:10452000ED91FC910190F081E02D0995C69586955D
:104530004C2F481B60E070E0C801F6010995D801D6
:10454000ED91FC91C484D584D7011796ED91FC912F
:10455000189786819781DC01ED91FC910190F081A3
:10456000E02D0995C82FD7011796ED91FC9118976A
:1045700084819581DC01ED91FC910190F081E02D29
:104580000995C69586954C2F481B60E070E0C801E0
:10459000F601CF911F910F91FF90EF90DF90CF9098
:1045A000099402970C946B22DC01CB01FC01F99970
:1045B000FECF06C0F2BDE1BDF89A319600B40D926F
:1045C00041505040B8F70895F999FECF92BD81BD92
:1045D000F89A992780B50895262FF999FECF1FBA2A
:1045E00092BD81BD20BD0FB6F894FA9AF99A0FBE1C
:1045F000019608955058BB27AA270E9412230C94B5
:104600008C240E947E2438F00E94852420F039F406
:104610009F3F19F426F40C947B240EF4E095E7FBFD
:104620000C947524E92F0E949D2458F3BA17620751
:1046300073078407950720F079F4A6F50C94BF243E
:104640000EF4E0950B2EBA2FA02D0B01B9019001AD
:104650000C01CA01A0011124FF27591B99F0593FF1
:1046600050F4503E68F11A16F040A22F232F342F39
:104670004427585FF3CF469537952795A795F04087
:104680005395C9F77EF41F16BA0B620B730B840B9C
:10469000BAF09150A1F0FF0FBB1F661F771F881F54
:1046A000C2F70EC0BA0F621F731F841F48F48795AC
:1046B00077956795B795F7959E3F08F0B0CF93959E
:1046C000880F08F09927EE0F9795879508950E9417
:1046D000512408F481E008950E9480230C948C24D6
:1046E0000E94852458F00E947E2440F029F45F3F08
:1046F00029F00C94752451110C94C0240C947B2443
:104700000E949D2468F39923B1F3552391F3951BDF
:10471000550BBB27AA2762177307840738F09F5FE2
:104720005F4F220F331F441FAA1FA9F335D00E2E4F
:104730003AF0E0E832D091505040E695001CCAF7BC
:104740002BD0FE2F29D0660F771F881FBB1F26177F
:1047500037074807AB07B0E809F0BB0B802DBF0156
:10476000FF2793585F4F3AF09E3F510578F00C9425
:1047700075240C94C0245F3FE4F3983ED4F38695EF
:1047800077956795B795F7959F5FC9F7880F911D46
:104790009695879597F90895E1E0660F771F881F32
:1047A000BB1F621773078407BA0720F0621B730BE5
:1047B000840BBA0BEE1F88F7E09508950E94E5235D
:1047C0006894B1110C94C02408950E94A52488F027
:1047D0009F5798F0B92F9927B751B0F0E1F0660FC5
:1047E000771F881F991F1AF0BA95C9F714C0B13006
:1047F00091F00E94BF24B1E008950C94BF24672F6C
:10480000782F8827B85F39F0B93FCCF38695779534
:104810006795B395D9F73EF490958095709561951D
:104820007F4F8F4F9F4F0895E89409C097FB3EF448
:1048300090958095709561957F4F8F4F9F4F9923ED
:10484000A9F0F92F96E9BB279395F695879577956B
:104850006795B795F111F8CFFAF4BB0F11F460FF2B
:104860001BC06F5F7F4F8F4F9F4F16C0882311F083
:1048700096E911C0772321F09EE8872F762F05C097
:10488000662371F096E8862F70E060E02AF09A9532
:10489000660F771F881FDAF7880F9695879597F927
:1048A0000895990F0008550FAA0BE0E8FEEF1616C1
:1048B0001706E807F907C0F012161306E407F50714
:1048C00098F0621B730B840B950B39F40A2661F088
:1048D000232B242B252B21F408950A2609F4A1402B
:1048E000A6958FEF811D811D089597F99F6780E838
:1048F00070E060E008959FEF80EC089500240A9432
:104900001616170618060906089500240A941216AA
:104910001306140605060895092E0394000C11F4DD
:10492000882352F0BB0F40F4BF2B11F460FF04C08A
:104930006F5F7F4F8F4F9F4F089557FD9058440FE3
:10494000551F59F05F3F71F04795880F97FB991FEE
:1049500061F09F3F79F087950895121613061406AB
:10496000551FF2CF4695F1DF08C016161706180638
:10497000991FF1CF86957105610508940895E89413
:10498000BB2766277727CB0197F908950E9451240A
:1049900008F48FEF08950E94DE240C948C240E946A
:1049A0007E2438F00E94852420F0952311F00C9489
:1049B00075240C947B2411240C94C0240E949D2403
:1049C00070F3959FC1F3950F50E0551F629FF00162
:1049D000729FBB27F00DB11D639FAA27F00DB11D7B
:1049E000AA1F649F6627B00DA11D661F829F222704
:1049F000B00DA11D621F739FB00DA11D621F839F8B
:104A0000A00D611D221F749F3327A00D611D231F60
:104A1000849F600D211D822F762F6A2F11249F57AE
:104A200050409AF0F1F088234AF0EE0FFF1FBB1FB1
:104A3000661F771F881F91505040A9F79E3F510570
:104A400080F00C9475240C94C0245F3FE4F3983EEE
:104A5000D4F3869577956795B795F795E7959F5F1A
:104A6000C1F7FE2B880F911D9695879597F90895AC
:104A700097FB072E16F4009407D077FD09D00E940B
:104A80004C2507FC05D03EF4909581959F4F0895E5
:104A9000709561957F4F0895AA1BBB1B51E107C01C
:104AA000AA1FBB1FA617B70710F0A61BB70B881FBE
:104AB000991F5A95A9F780959095BC01CD0108954D
:104AC000EE0FFF1F0590F491E02D09940F931F93B3
:104AD000CF93DF938230910510F482E090E0E09173
:104AE0003303F091340320E030E0A0E0B0E03097F1
:104AF00019F1408151810281138148175907C8F08B
:104B00008417950769F4109731F012960C93129759
:104B100013961C9327C0009333031093340322C0D1
:104B20002115310519F04217530718F49A01BD01F8
:104B3000EF01DF01F801DBCF21153105F9F0281B6A
:104B4000390B2430310580F48A819B816115710510
:104B500021F0FB019383828304C0909334038093FC
:104B60003303FE01329644C0FE01E20FF31F81932E
:104B7000919322503109398328833AC0209131031F
:104B800030913203232B41F420911501309116010D
:104B9000309332032093310320911301309114019B
:104BA0002115310541F42DB73EB7409117015091C1
:104BB0001801241B350BE0913103F0913203E21709
:104BC000F307A0F42E1B3F0B2817390778F0AC0130
:104BD0004E5F5F4F2417350748F04E0F5F1F50930D
:104BE0003203409331038193919302C0E0E0F0E0FF
:104BF000CF01DF91CF911F910F910895CF93DF9354
:104C0000009709F481C0FC01329713821282A091AF
:104C10003303B0913403109781F420813181820FE6
:104C2000931F20913103309132032817390751F532
:104C3000F0933203E093310367C0ED0120E030E0F0
:104C4000CE17DF0740F44A815B819E014115510573
:104C5000F1F0EA01F5CFD383C28340815181840F03
:104C6000951FC817D90759F488819981840F951F1A
:104C70000296918380838A819B819383828321150D
:104C8000310529F4F0933403E09333033DC0E90187
:104C9000FB83EA8349915991C40FD51FEC17FD0797
:104CA00061F480819181840F951F0296E9019983B7
:104CB0008883828193819B838A83E0E0F0E012966F
:104CC0008D919C911397009719F0FD01DC01F7CFAE
:104CD0008D919C9111979D012E5F3F4F820F931FE5
:104CE00020913103309132032817390769F4309746
:104CF00029F4109234031092330302C013821282FB
:104D0000B0933203A0933103DF91CF91089581E0F6
:104D100090E0F8940C949326DC0101C06D9341500F
:0A4D20005040E0F70895F894FFCF2B
:104D2A000C005009000300000000000101400300CC
:104D3A00400301000035038000A59E8C000000009E
:104D4A0070026D02FE060207E902DF02D702C902FB
:104D5A00BD02790273027E0200000000000000001A
:104D6A00B500B500B500B500B500B500B500B50091
:104D7A000080808080800000020200000000B408E9
:104D8A00FC0636056802600258023B022F02250221
:104D9A001C020000000006156B227D185E1DFEFF36
:104DAA000000D12200000000E31900000000FA0E02
:104DBA00000000004810000000001A130000000064
:104DCA00961100000000E41200000000D418000050
:104DDA000000B50000807F7F7F7F00000000000098
:104DEA00F40200000000BB1796170000000011171C
:104DFA00DE160000000055183D1800000000641877
:104E0A00641800000000C1008700D501DA07060215
:104E1A00E401F80100000000391B001011121314FC
:104E2A001516171718191A1B1B1C1D1E1E1F2021C9
:104E3A002222232424252626272828292A2A2B2CFD
:104E4A002C2D2D2E2F2F303031313233333434354F
:104E5A00353636373738383839393A3A3B3B3B3CBE
:104E6A003C3D3D3D3E3E3F3F3F4040404041414149
:104E7A0042424243434343434444444444454545F0
:104E8A0045454646464646464646464647474747B6
:0A4E9A004747474747474747474748
:00000001FF
